:020000040000FA
:10000000FF3FFF3FE322E32285019F1686018B011C
:10001000103065007C3066002730620014309C0090
:100020009D099F1A8D21A5222E219A229F123230DE
:10003000E5229B2122201D081102031D6F229C0B2B
:10004000172807281430940006093C3903190800C2
:100050008400E322792206093C3903194728940BCE
:1000600028288A01840C840C0F30040582070800BC
:10007000402940295A287A284C284C28080037293A
:10008000080008000800F528080008000800041906
:100090006A2984197B292029FF308C008D008F006C
:1000A0009000E530041CBE308E009F11041C9F158B
:1000B0009F228429FF308C008D008F009000AF229A
:1000C0009A00F039A03C031D71280F3088050808FC
:1000D0008E00080E88070A300E021A3003198E00AF
:1000E00077280F308805A03088071A308E00AC22A0
:1000F0007922842991019201930106308400910AAA
:100100000F3011050A3CF03003199105A02085211C
:10011000A020061E8D28E32288280A309400061AA3
:100120007F28E322940B8F28840B9728AA28043079
:100130009A000310910D920D930D9A0B99287F2828
:10014000110897001208980013089900FF309B00CF
:100150002A22792A06309A00970198019901D22023
:1001600011080F399B000319C528160899071508AF
:1001700098070318990A14089707031CC32801302D
:100180009807031899079B0BB52804309B000310B0
:10019000930C920C910C9B0BC7289A0BAF28C4228E
:1001A0006F2284298A01DA209400E3209500EC2054
:1001B000960008001A0882070000A0341034E834C2
:1001C00064340A3401341A08820700008634273464
:1001D00003340034003400341A088207000001346C
:1001E000003400340034003400349F17022185218C
:1001F000061D1329861D1729061E1B29861E1B296D
:100200000221F8289B211E089400950196010722DF
:100210000D0EF03990000C0E0F3990070C0EF039CE
:100220008F006F22E32A9E0F00299E0A00299E0B51
:1002300000299E0300290F309F0595226F228429F3
:10024000041E28291F1C26291F102D291F142D29A3
:100250009F1C2C299F102D299F149F229F18051445
:100260009F1C05101F1886171F1C861308001F1DD2
:100270003B291F113C291F159F226F229F22842991
:10028000B222AF220F399400950090000A3C1A3038
:10029000031990009B0C9A0C970C960C940B4A290E
:1002A0009713041897170130971FF1308E00960DA1
:1002B000970D9A0D9B0D950B57293B3089001B0814
:1002C0008800D722890A1A088800D7228C018D015C
:1002D0008F018429AF229A009B009B0E0F309A0554
:1002E0001B051A02031908000A301A020319080034
:1002F000880AAC228D29AF220F399A001A0B812966
:1003000008008803AC228D298D217922E322060979
:100310003C39031D85299D090800AF2285140F393A
:100320009A0085109A0B9529080005150000051103
:100330009A0B952908001E0884008B019301810106
:1003400046309B00831685158312B8309A009A0BAD
:10035000A729E0219B0BA5290000840BAC29E021F3
:100360008511831685118312E02101089200910105
:100370008515910A85110000010812020319B82998
:10038000910A9109910A910A0310930C920C910C15
:100390000310930C920C910C9F1B08009F19DD29F0
:1003A000061F0800AF220F398400B2229B0C9A0C62
:1003B000840BD629031CE729F729061FE729F7290B
:1003C0000B1DE5290B11930A080000000800BA2252
:1003D0001908930218089202031C9303170891024C
:1003E0000318080001309202031C93020800BA228D
:1003F00019089307180892070318930A170891071A
:10040000031C0800013092070318930708009701A6
:100410009801990114309A00170865229707170868
:100420006A22970718086522980718086A22980711
:1004300019086522990719086A229907940D950DE4
:10044000960D970D980D990D1710161A17149A0BF3
:100450000C2A9B015022502250225022502250221E
:100460009F1B0800B03090001F19422A0E0E0F3952
:100470008F000F308E058E0E0D0E0F398E070F3048
:100480008D0508000E088F000D0E0F398E000D0E21
:10049000F0398D000C0E0F398D070F308C050800D8
:1004A00004309A00970D980D990D8C0D8D0D8E0DC1
:1004B0009A0B522A0C080F39003003190A30031D19
:1004C0001B141B1C00308C0708000F39043C031858
:1004D00000340334F0394F3C031800343034110831
:1004E0009D00110894001208950013089600072239
:1004F000792AFC3086058316811728309A00901BD4
:100500008614901F86108C0D06148D0D8E0D8F0D88
:10051000900D06109A0B7F2A86108C0D8D0D81137D
:100520008E0D8F0D900D831208003D3089001E083E
:100530008800D72A3D308900D0229E0008003E3036
:1005400089001F080F398800D72A3E308900D02241
:100550000F399F00080088003F308900D72A3F30BC
:100560008900D02A3B308900D0229B00890AD02202
:100570009A0008008901D0229900890AD0229800A7
:10058000890AD02297000800890119088800D7221B
:10059000890A18088800D722890A17088800D72AEC
:1005A000831608140818D22A831208080800831634
:1005B000081555308900AA30890088148818DE2A69
:1005C0000811831208008312B6309B009A009A0B20
:1005D000E72A9B0BE62A0800FF3FFF3FFF3FFF3F54
:1005E000FF3FFF3FFF3FFF3FFF3FFF3FFF3FFF3F1B
:1005F000FF3FFF3FFF3FFF3FFF3FFF3FFF3FFF3F0B
:10060000FF3FFF3FFF3FFF3FFF3FFF3FFF3FFF3FFA
:10061000FF3FFF3FFF3FFF3FFF3FFF3FFF3FFF3FEA
:10420000000000000000FF00FF00FF00FF00FF00B3
:10421000FF00FF00FF00FF00FF00FF00FF00FF00A6
:10422000FF00FF00FF00FF00FF00FF00FF00FF0096
:10423000FF00FF00FF00FF00FF00FF00FF00FF0086
:10424000FF00FF00FF00FF00FF00FF00FF00FF0076
:10425000FF00FF00FF00FF00FF00FF00FF00FF0066
:10426000FF00FF00FF00FF00FF00FF00FF00FF0056
:10427000FF00FF00FF00FF00FF0080000000A10022
:08400000FF3FFF3FFF3FFF3FC0
:02400E00F93F78
:00000001FF
